:100000001201C31201D575E0811201B675E020120C
:1000100001A975E0201201A975E0201201A975E07F
:10002000201201A975E0381201A975E0301201A96A
:1000300075E0351201A975E0311201A975E02012B1
:1000400001A975E0201201A975E0441201A975E02B
:10005000691201A975E0631201A975E0651201A991
:1000600075E0C01201B675E0481201A975E06F1283
:1000700001A975E06C1201A975E0641201A975E08F
:10008000201201A975E0501201A975E0331201A9EF
:1000900075E02E1201A975E0351201A975E0201254
:1000A00001A975E0621201A975E0751201A975E058
:1000B000741201A975E0741201A975E06F1201A90B
:1000C00075E06E1201A920B5FD75E0C01201B6758C
:1000D000E06F1201A975E06E1201A975E0651201C9
:1000E000A9780D1201A020B5FD75E0C01201B6750A
:1000F000E0741201A975E0771201A975E06F120191
:10010000A9780D1201A020B5FD75E0C01201B675E9
:10011000E0741201A975E0681201A975E07212017C
:10012000A975E0651201A975E0651201A9780B12A5
:1001300001A020B5FD75E0C01201B675E0661201A0
:10014000A975E06F1201A975E0751201A975E07239
:100150001201A9780C1201A020B5FD75E0C01201B2
:10016000B675E0661201A975E0691201A975E0761D
:100170001201A975E0651201A9780C1201A020B541
:10018000FD75E0C01201B675E0731201A975E06952
:100190001201A975E0781201A9780D1201A001C61B
:1001A00075E0201201A9D8F822D29285E0A0D29061
:1001B000C2901201DB22C29285E0A0D290C29012BE
:1001C00001DB22C29175E03831B675E00E31B675AB
:1001D000E00631B62275E00131B6227CFFDCFE225A
:00000001FF
